:100000000C9452000C946F000C946F000C946F00D1
:100010000C946F000C946F000C946F000C946F00A4
:100020000C946F000C946F000C946F000C946F0094
:100030000C946F000C946F000C946F000C946F0084
:100040000C94B4000C946F000C946F000C946F002F
:100050000C946F000C946F000C946F000C946F0064
:100060000C946F000C946F00000000002500280025
:100070002B0000000000240027002A0004040404D0
:100080000404040402020202020203030303030342
:10009000010204081020408001020408102001021F
:1000A0000408102011241FBECFEFD8E0DEBFCDBF63
:1000B00011E0A0E0B1E0E0EEF4E002C005900D92A6
:1000C000A030B107D9F721E0A0E0B1E001C01D9256
:1000D000AD30B207E1F70E94FE000C946E020C9462
:1000E0000000CF93DF9390E0FC01E057FF4F249195
:1000F00084589F4FFC0184918823D1F090E0880FB1
:10010000991FFC01EE58FF4FA591B491FC01E859ED
:10011000FF4FC591D49161110EC09FB7F8948C9197
:10012000E22FE0958E238C932881E223E8839FBF02
:10013000DF91CF9108958FB7F894EC91E22BEC9377
:100140008FBFF6CF8E50806480937C0080917A00C0
:10015000806480937A0080917A0086FDFCCF809144
:1001600078009091790008951F920F920FB60F9228
:1001700011242F933F938F939F93AF93BF938091BD
:10018000090190910A01A0910B01B0910C013091ED
:10019000080123E0230F2D3758F50196A11DB11D4D
:1001A000209308018093090190930A01A0930B0109
:1001B000B0930C018091040190910501A09106017A
:1001C000B09107010196A11DB11D80930401909388
:1001D0000501A0930601B0930701BF91AF919F91D4
:1001E0008F913F912F910F900FBE0F901F901895F8
:1001F00026E8230F0296A11DB11DD2CF789484B5B5
:10020000826084BD84B5816084BD85B5826085BD12
:1002100085B5816085BD80916E00816080936E00A0
:100220001092810080918100826080938100809192
:100230008100816080938100809180008160809343
:1002400080008091B10084608093B1008091B00003
:1002500081608093B00080917A00846080937A00FE
:1002600080917A00826080937A0080917A00816028
:1002700080937A0080917A00806880937A0010924F
:10028000C10061E08AE00E94710061E08BE00E94A1
:10029000710061E083E00E94710060E081E10E94F2
:1002A000710060E082E10E94710060E08FE00E94D6
:1002B000710060E080E10E94710010928000109255
:1002C000810081EA8093800089E080938100109210
:1002D0008B0010928A001092B0001092B10083EA55
:1002E0008093B00081E08093B1001092B30010922F
:1002F000B400FF24F39470E0A72E70E0B72E8EE0D8
:100300000E94A20010E087369105A4F011E0853329
:1003100021E092077CF012E0833042E0940754F031
:1003200013E0813D22E092072CF014E08F399340D6
:100330000CF015E08FE00E94A2006C0181E10E94A8
:10034000A200AC01C601DD0CAA0BBB0B052E000CF4
:10035000660B770B840F951FA61FB71FD0E0C0E078
:10036000B7FD08C0EC0181159440A105B10514F05A
:10037000CFEFD3E080E10E94A2006C0182E10E94F5
:10038000A200AC01C601DD0CAA0BBB0B052E000CB4
:10039000660B770B840F951FA61FB71FB7FD31C0E3
:1003A000811544E09407A105B10574F531E0C13031
:1003B00022E0D2070CF430E021E0813042E09407E3
:1003C0000CF420E0133009F461C008F5113009F491
:1003D0004FC0123009F457C0C13022E0D2072CF0D0
:1003E000813042E094070CF04AC0C130D24024F082
:1003F000813092400CF051C04FEF50E030E020E0EF
:100400005EC090E080E0D2CF8FEF93E0CFCF14308A
:1004100009F445C0153001F7C130D2404CF040918D
:100420000301411105C0409102014F254093020193
:10043000813092404CF080910101811105C0809182
:1004400000018F2580930001309303012093010167
:10045000809102012FEF30E0811102C030E020E0F6
:10046000809100014FEF50E0811129C040E027C08A
:10047000C130D24024F4813092400CF4BDCF40E032
:100480002FEF30E01CC03213FACFB6CF8C179D0788
:10049000B4F3C817D9070CF4AFCF40E0AFCFAC012D
:1004A00055954795559547959E01359527953595D1
:1004B00027958C179D071CF0922F9A01492F309396
:1004C0008B0020938A004093B3002093B400A114C2
:1004D000B10409F414CF0E94000011CFF894FFCFAB
:00000001FF
